:1000000045C0000060C000005EC0000063C1000089
:100010005AC0000058C0000056C0000054C0000084
:1000200052C00000B6C100004EC000004CC000002D
:100030004AC0000048C0000046C0000044C00000A4
:1000400042C0000040C000003EC000003CC00000B4
:100050003AC0000038C0000036C0000034C00000C4
:1000600032C0000030C000002EC000002CC00000D4
:100070002AC0000028C0000026C0000024C00000E4
:1000800022C0000020C000001EC0000011241FBEBE
:10009000CFEFD0E1DEBFCDBF11E0A0E0B1E0E8E1FD
:1000A000FDE000E00BBF02C007900D92AA32B1073D
:1000B000D9F721E0AAE2B1E001C01D92A633B20750
:1000C000E1F72FD127C69CCF9BB321E030E002C0DF
:1000D000220F331F8A95E2F7292B2BBB08959BB380
:1000E00021E030E002C0220F331F8A95E2F720950D
:1000F00029232BBB089586E090E0E6DF83EC99E0AE
:100100000197F1F700C0000086E090E0E8DF87E8A3
:1001100093E10197F1F700C000000895CF93C82F35
:1001200085BB84E090E0D0DFE6DFC295C07FC5BB31
:1001300084E090E0C9DFDFDFCF910895CF93C82F2F
:1001400085BB84E090E0CBDFD6DFC295C07FC5BB26
:1001500084E090E0C4DFCFDFCF91089581E0EEDF4F
:1001600087E893E10197F1F700C0000080E8E6CF4F
:100170000895CF938FEF84BB85BB8ABB15BA1BBA9A
:10018000C0E2C5BBB8DFC5BBB6DF80E885BBB3DF67
:1001900015BAB1DF80EF85BBAEDF15BAACDF80E604
:1001A00085BBA9DF82E0CADFA6DFCF910895CF9398
:1001B000DF93EC0102C0B2DF219688818111FBCF71
:1001C000DF91CF9108954F925F926F927F928F92BD
:1001D0009F92AF92BF92CF92DF92EF92FF920F93D6
:1001E0001F93CF93DF93CDB7DEB7D82EC92E942EB1
:1001F000852E762E672E522E432EADB6BEB63F9379
:100200002F937F936F935F934F939F938F930F2EB3
:10021000F5E1EF2EF1E0FF2EF02DFF92EF921F920D
:100220001F921F921F928DD201962DB73EB7225F6B
:100230003F4F0FB6F8943EBF0FBE2DBF281B390BA2
:100240000FB6F8943EBF0FBE2DBF0DB71EB70F5FA0
:100250001F4F4F925F926F927F928F929F92CF9299
:10026000DF92FF92EF929F938F931F930F9369D228
:10027000802F912F9CDF8DB79EB70E960FB6F89406
:100280009EBF0FBE8DBF0FB6F894BEBE0FBEADBEF3
:10029000DF91CF911F910F91FF90EF90DF90CF9062
:1002A000BF90AF909F908F907F906F905F904F9096
:1002B000089520910001222351F00197439738F4CB
:1002C000D7D01092000161E080E092E0C4C00895B0
:1002D0000AC108951F920F920FB60F9211240BB608
:1002E0000F922F933F934F935F936F937F938F93CF
:1002F0009F93AF93BF93EF93FF9302D1FF91EF9141
:10030000BF91AF919F918F917F916F915F914F912D
:100310003F912F910F900BBE0F900FBE0F901F902B
:100320001895D2D026DFA6D088E691E02DD089E5B9
:1003300091E004D187EA91E60197F1F700C000004F
:100340000DDF60E088E592E086D008DFFCD0AB01ED
:10035000BC0121E231E084E291E035DF84E690E007
:10036000A4D0F3CF90913101911107C0E82FF0E0B4
:10037000EF5FFE4F808183B90895E82FF0E0E75FDB
:10038000FE4F808183B908959093330180933201A9
:1003900008951F920F920FB60F9211240BB60F9271
:1003A0002F933F934F935F936F937F938F939F937D
:1003B000AF93BF93EF93FF9314BC80912A01D2DFD8
:1003C00080912A01873020F48F5F80932A0130C00A
:1003D00010922A0180912B0190912C01009799F4A1
:1003E00080913101811104C081E08093310102C00C
:1003F0001092310180912D0190912E0190932C014A
:1004000080932B0115C09C012F713327232B39F4C6
:10041000E0913201F0913301309709F00995809114
:100420002B0190912C01019790932C0180932B012B
:10043000FF91EF91BF91AF919F918F917F916F91BC
:100440005F914F913F912F910F900BBE0F900FBE78
:100450000F901F90189590932C0180932B019093EF
:100460002E0180932D01609331018CE085BD0895AC
:1004700015BC08958FEF82B98093640081E080936A
:10048000650013B886E983BD80E887BF7894089536
:1004900020E030E006C043E04A95F1F700002F5F0E
:1004A0003F4F28173907B8F3089520E030E008C01F
:1004B000E3ECF9E03197F1F700C000002F5F3F4F08
:1004C00028173907A8F308958FEF8093640011BAB5
:1004D00080E380936A0089B7846089BF1FBC8CE089
:1004E0008EBD78940895CF93DF93C5E6D0E018824F
:1004F0008AE090E0CDDF81E08883DF91CF9108959D
:1005000080911101813041F480E280936A001DBC2A
:100510001CBC10921101089580E380936A008CB591
:100520009DB59093300180932F01E0913401F091BB
:100530003501099581E0809311010895909335016B
:1005400080933401089560912F017091300180E013
:1005500090E006D020E030E04AE253E43EC0089547
:10056000E89409C097FB3EF490958095709561954D
:100570007F4F8F4F9F4F9923A9F0F92F96E9BB2703
:100580009395F695879577956795B795F111F8CF7F
:10059000FAF4BB0F11F460FF1BC06F5F7F4F8F4FEA
:1005A0009F4F16C0882311F096E911C0772321F0E0
:1005B0009EE8872F762F05C0662371F096E8862F78
:1005C00070E060E02AF09A95660F771F881FDAF7CF
:1005D000880F9695879597F908950BD078C069D0C4
:1005E00028F06ED018F0952309F05AC05FC011248E
:1005F000A2C07ED0A0F3959FD1F3950F50E0551F78
:10060000629FF001729FBB27F00DB11D639FAA2767
:10061000F00DB11DAA1F649F6627B00DA11D661FB6
:10062000829F2227B00DA11D621F739FB00DA11DD7
:10063000621F839FA00D611D221F749F3327A00D91
:10064000611D231F849F600D211D822F762F6A2F2D
:1006500011249F5750408AF0E1F088234AF0EE0FB2
:10066000FF1FBB1F661F771F881F91505040A9F7BF
:100670009E3F510570F014C05EC05F3FECF3983EA2
:10068000DCF3869577956795B795F795E7959F5F26
:10069000C1F7FE2B880F911D9695879597F90895C0
:1006A00097F99F6780E870E060E008959FEF80EC25
:1006B000089500240A9416161706180609060895C8
:1006C00000240A9412161306140605060895092E2E
:1006D0000394000C11F4882352F0BB0F40F4BF2B9D
:1006E00011F460FF04C06F5F7F4F8F4F9F4F0895DD
:1006F00057FD9058440F551F59F05F3F71F04795D3
:10070000880F97FB991F61F09F3F79F087950895B7
:10071000121613061406551FF2CF4695F1DF08C0D6
:10072000161617061806991FF1CF869571056105F3
:1007300008940895E894BB2766277727CB0197F99B
:1007400008950F931F93CF93DF93CDB7DEB72E9706
:100750000FB6F894DEBF0FBECDBF0D891E898F89FD
:10076000988D26E02C831A83098397FF02C080E0CE
:1007700090E801979E838D83AE01455E5F4F698D42
:100780007A8DCE01019619D04D815E8157FD0AC048
:100790002F813885421753070CF49A01F801E20FB4
:1007A000F31F10822E960FB6F894DEBF0FBECDBF9A
:1007B000DF91CF911F910F9108952F923F924F9209
:1007C0005F926F927F928F929F92AF92BF92CF92E1
:1007D000DF92EF92FF920F931F93CF93DF93CDB7EA
:1007E000DEB72B970FB6F894DEBF0FBECDBF6C01FE
:1007F0007B018A01FC0117821682838181FFBFC1C0
:10080000CE0101963C01F6019381F70193FD85919C
:1008100093FF81917F01882309F4ADC1853239F4BA
:1008200093FD859193FF81917F01853221F4B6017B
:1008300090E0D6D1E8CF912C212C312CFFE1F3159B
:10084000D8F08B3279F038F4803279F08332A1F429
:10085000232D20611DC08D3261F0803369F4232D7A
:10086000216016C0832D8260382EE32DE4603E2E79
:100870002AC0F32DF8601DC037FC2DC020ED280FD5
:100880002A3040F08E32B9F436FC75C1232D206435
:10089000322E19C036FE06C08AE0989E200D112423
:1008A000922E11C0EAE02E9E200D1124222EF32D4F
:1008B000F0623F2E08C08C3621F4832D8068382EDC
:1008C00002C0883641F4F70193FD859193FF819131
:1008D0007F018111B3CF982F9F7D9554933028F4D9
:1008E0000C5F1F4F9FE399830DC0833631F0833730
:1008F00071F0833509F055C020C0F80180818983EB
:100900000E5F1F4F88248394912C530112C028013D
:10091000F2E04F0E511CF801A080B18036FE03C0FA
:10092000692D70E002C06FEF7FEFC5014ED14C0121
:100930008201F32DFF773F2E15C0280122E0420EE1
:10094000511CF801A080B18036FE03C0692D70E013
:1009500002C06FEF7FEFC5012DD14C01F32DF06880
:100960003F2E820133FC19C0822D90E08816990633
:10097000A0F4B60180E290E033D12A94F5CFF501DE
:1009800037FC859137FE81915F01B60190E028D157
:1009900021102A9421E0821A91088114910479F798
:1009A000E1C0843611F0893639F5F80137FE07C009
:1009B00060817181828193810C5F1F4F08C06081CB
:1009C0007181072E000C880B990B0E5F1F4FF32DC2
:1009D000FF763F2E97FF09C09095809570956195A1
:1009E0007F4F8F4F9F4FF0683F2E2AE030E0A301EA
:1009F00033D1882E861844C0853731F4232D2F7EBD
:100A0000B22E2AE030E025C0932D997FB92E8F3683
:100A1000C1F018F4883579F0AEC0803719F0883706
:100A200021F0A9C0E92FE061BE2EB4FE0DC0FB2D60
:100A3000F460BF2E09C034FE0AC0292F2660B22EF2
:100A400006C028E030E005C020E130E002C020E12F
:100A500032E0F801B7FE07C0608171818281938125
:100A60000C5F1F4F06C06081718180E090E00E5FD7
:100A70001F4FA301F1D0882E8618FB2DFF773F2E44
:100A800036FE0DC0232D2E7FA22E891458F434FE7D
:100A90000BC032FC09C0832D8E7EA82E05C0B82C59
:100AA000A32C03C0B82C01C0B92CA4FE0FC0FE01BA
:100AB000E80DF11D8081803321F49A2D997EA92EB5
:100AC00009C0A2FE06C0B394B39404C08A2D8678F0
:100AD00009F0B394A3FC10C0A0FE06C0B21480F4C9
:100AE000280C922C9B180DC0B21458F4B60180E269
:100AF00090E076D0B394F8CFB21418F42B1802C05B
:100B0000982C212CA4FE0FC0B60180E390E068D0A1
:100B1000A2FE16C0A1FC03C088E790E002C088E5F1
:100B200090E0B6010CC08A2D867851F0A1FE02C07B
:100B30008BE201C080E2A7FC8DE2B60190E050D0CC
:100B4000891430F4B60180E390E04AD09A94F8CF4B
:100B50008A94F301E80DF11D8081B60190E040D048
:100B60008110F6CF222009F44ECEB60180E290E04B
:100B700037D02A94F7CFF6018681978102C08FEF94
:100B80009FEF2B960FB6F894DEBF0FBECDBFDF915F
:100B9000CF911F910F91FF90EF90DF90CF90BF907A
:100BA000AF909F908F907F906F905F904F903F900D
:100BB0002F900895FC010590615070400110D8F706
:100BC000809590958E0F9F1F0895FC016150704095
:100BD00001900110D8F7809590958E0F9F1F089572
:100BE0000F931F93CF93DF93FB01238121FD03C05C
:100BF0008FEF9FEF2CC022FF16C0468157812481C2
:100C000035814217530744F4A081B1819D012F5FC4
:100C10003F4F318320838C93268137812F5F3F4F55
:100C20003783268314C08B01EC01FB010084F1851E
:100C3000E02D0995892BE1F6D80116968D919C91AE
:100C40001797019617969C938E931697CE01DF9176
:100C5000CF911F910F910895FA01AA27283051F1E1
:100C6000203181F1E8946F936E7F6E5F7F4F8F4FDD
:100C70009F4FAF4FB1E03ED0B4E03CD0670F781F3C
:100C8000891F9A1FA11D680F791F8A1F911DA11D21
:100C90006A0F711D811D911DA11D20D009F468945A
:100CA0003F912AE0269F11243019305D3193DEF602
:100CB000CF010895462F4770405D4193B3E00FD0B8
:100CC000C9F7F6CF462F4F70405D4A3318F0495DA3
:100CD00031FD4052419302D0A9F7EACFB4E0A69586
:100CE0009795879577956795BA95C9F700976105A8
:100CF000710508959B01AC010A2E069457954795FE
:100D000037952795BA95C9F7620F731F841F951FF2
:080D1000A01D0895F894FFCF27
:100D180001080C0406020301090901030206040C78
:100D2800080125640025733A20252E336620257393
:0A0D380000636D006469737400002D
:00000001FF
